:100000000C944B000C9466000C9466000C946600F3
:100010000C9466000C9466000C9466000C946600C8
:100020000C9466000C9466000C9466000C946600B8
:100030000C9466000C9466000C9466000C946600A8
:100040000C9466000C9466000C9466000C94660098
:100050000C946600202078782E7878782E78782096
:100060004D487A203A312020202020202020444C66
:10007000354E4547004672657175656E6379636FED
:10008000756E74657256657220312E3120202044C1
:100090004C354E45470011241FBECFE5D4E0DEBFEE
:1000A000CDBF10E0A0E6B0E0EEE7FEE002C00590B4
:1000B0000D92A636B107D9F710E0A6E6B0E001C070
:1000C0001D92A838B107E1F70C9418030C940000B6
:1000D000AC0183E083BF20E030E02417350768F4EB
:1000E00096EC92BF88B7816088BF08B600FEFDCF4E
:1000F0002F5F3F4F24173507A0F3089580916600C6
:100100008F5F80936600853010F0109266008091BA
:100110006600882361F481E38093780080E2809315
:10012000790080937A0080937B008DE43DC081301C
:1001300051F486E38093780084E38093790080E231
:1001400080937A000CC08230A9F481E38093780018
:1001500082E38093790088E380937A0080E2809341
:100160007B0087E4809373008EE280936A00809323
:100170006E0021C0833059F486E38093780084E3D5
:100180008093790080E380937A0080E20AC0843013
:1001900091F481E38093780080E3809379008093E9
:1001A0007A0080937B0087E4809373008EE28093D3
:1001B0006B0080936F0088EC90E00E9468000895C7
:1001C00098B39F7098BB982F907F88B3892B88BB7A
:1001D000959A959881E090E00E94680008951F9399
:1001E000CF93DF93969880E80E94E00080E00E9421
:1001F000E0008FE090E00E946800969AC7E6D0E0A9
:100200001FE08881807F0E94E00089918295807F35
:100210000E94E000115017FFF4CF969880EC0E94E6
:10022000E00080E00E94E0008FE090E00E94680023
:10023000969AC7E7D0E01FE08881807F0E94E000A7
:1002400089918295807F0E94E000115017FFF4CFC2
:10025000DF91CF911F910895CF938FE090E00E949E
:10026000680082B38F7982BBC2E080E30E94E00025
:1002700085E090E00E946800C150C7FFF6CF80E2A1
:100280000E94E00085E090E00E94680080E20E9409
:10029000E00080E80E94E00085E090E00E946800B5
:1002A00080E00E94E00080E10E94E00085E090E0B4
:1002B0000E94680080E00E94E00080E60E94E0006A
:1002C00085E090E00E94680080E00E94E00080EC01
:1002D0000E94E00085E090E00E946800CF910895C0
:1002E000EF92FF920F931F93CF93DF93CDB7DEB7BB
:1002F00064970FB6F894DEBF0FBECDBF7B018C01B3
:1003000080916600882309F03FC0C801B70124E648
:1003100030E040E050E00E94FE067B018C0137E0B7
:1003200016950795F794E7943A95D1F71F930F9395
:10033000FF92EF9280E690E09F938F93CE0101961B
:100340009F938F930E9477038981809368008A81AD
:10035000809369008B8180936A008C8180936C000C
:100360008D8180936D008E8180936E008F8180934C
:1003700070008885809371008DB79EB708960FB680
:10038000F8949EBF0FBE8DBF80916600813079F5D5
:1003900016950795F794E7941F930F93FF92EF92AA
:1003A00080E690E09F938F93CE0101969F938F9369
:1003B0000E9477038A81809369008B8180936B0010
:1003C0008C8180936C008D8180936D008E818093F1
:1003D0006F008F81809370008885809371008DB746
:1003E0009EB708960FB6F8949EBF0FBE8DBF809142
:1003F0006600823059F51F930F93FF92EF9280E6CB
:1004000090E09F938F93CE0101969F938F930E94CC
:1004100077038A81809369008B8180936B008C8144
:1004200080936C008D8180936D008E8180936F002E
:100430008F81809370008885809371008DB79EB7FF
:1004400008960FB6F8949EBF0FBE8DBF80916600D0
:10045000833091F516950795F794E7941F930F93C2
:10046000FF92EF9280E690E09F938F93CE010196EA
:100470009F938F930E9477038981809368008A817C
:10048000809369008B8180936A008C8180936C00DB
:100490008D8180936D008E8180936E008F8180931B
:1004A00070008885809371008DB79EB708960FB64F
:1004B000F8949EBF0FBE8DBF80916600843009F016
:1004C0003FC0C801B70124E630E040E050E00E94A0
:1004D000FE067B018C0187E016950795F794E7945B
:1004E0008A95D1F71F930F93FF92EF9280E690E0E9
:1004F0009F938F93CE0101969F938F930E947703D2
:100500008981809368008A81809369008B818093C0
:100510006A008C8180936C008D8180936D008E8148
:1005200080936E008F818093700088858093710026
:100530008DB79EB708960FB6F8949EBF0FBE8DBFBD
:100540000E94EF0064960FB6F894DEBF0FBECDBFD9
:10055000DF91CF911F910F91FF90EF900895805DF3
:100560008A3308F0895F99270895EF92FF920F93DD
:100570001F937B018C01DC01CB012CE1B695A79583
:10058000979587952A95D1F78F700E94AF02809337
:100590007F00812F9927AA27BB278F700E94AF0267
:1005A00080938000D801C701E4E1B695A79597959F
:1005B0008795EA95D1F78F700E94AF0280938100F2
:1005C000C801AA27BB278F700E94AF0280938200C8
:1005D000D801C7016CE0B695A795979587956A9560
:1005E000D1F78F700E94AF0280938300BB27A12FA9
:1005F000902F8F2D8F700E94AF0280938400D801BE
:10060000C70144E0B695A795979587954A95D1F788
:100610008F700E94AF02809385008E2D8F700E9494
:10062000AF02809386001F910F91FF90EF90089585
:10063000CFE5D4E0DEBFCDBF86E08EBD8A9A80EFE5
:1006400087BB81B3806681BB939A979A0E942C01E5
:1006500065E770E087E690E00E94A8030E94EF0043
:1006600080ED97E00E94680064E570E087E690E026
:100670000E94A8030E94EF00849BFECF8499FECFC6
:1006800081E090E00E94680026B322702295220F3C
:10069000220F207C83B38F77282B8CB5482F5527CA
:1006A0008DB599277C01002711278701FF24EE24AF
:1006B000942F8827AA27BB27E80EF91E0A1F1B1FA5
:1006C000E20EF11C011D111D879904C0C801B7017C
:1006D0000E94B502C801B7010E947001929A9298D7
:1006E0001DBC1CBC8399C8CF0E947E00C5CF0F9350
:1006F0001F93CF93DF93CDB7DEB72C970FB6F89447
:10070000DEBF0FBECDBF0B891C89AD89BE8936E027
:100710003C8309831A838FEF9FE78D839E83AE010D
:10072000495E5F4FBD01CE0101960E94AF032F814C
:100730003885020F131FF80110822C960FB6F8941B
:10074000DEBF0FBECDBFDF91CF911F910F910895F6
:10075000FB01DC0105900D920020E1F708952F9236
:100760003F924F925F926F927F928F929F92AF9241
:10077000BF92CF92DF92EF92FF920F931F93CF938E
:10078000DF93CDB7DEB762970FB6F894DEBF0FBE2A
:10079000CDBFAA24BB2465014C011B014D875E8798
:1007A00044245524FC0146825782838181FDACC2DA
:1007B0008FEF9FEFB8C20894211C311C40FE92C2FB
:1007C000862D80538A30F0F4F0E36F1651F42A89B5
:1007D000222339F443FC05C080E091E0482A592ADD
:1007E00093C28AE09A89989F902D1124892F860DB3
:1007F00080538A8B882314F4EFE7EA8B43FC84C28E
:100800007A8882C243FE05C0FA89FF2311F421E0F1
:100810002A8B862D992787FD9095883691057CF542
:10082000853691050CF070C08335910509F49FC0A1
:1008300084359105BCF48B32910509F447C08C32A4
:10084000910544F48032910509F444C0839709F47A
:100850004BC03EC28D32910509F441C08E9709F418
:1008600048C036C28336910509F458C084369105D4
:100870000CF09AC08835910509F4D1C029C280379F
:10088000910509F4C4C08137910584F48C36910533
:10089000B1F18D3691052CF48936910509F484C0A7
:1008A00017C28F36910509F4AFC012C28537910582
:1008B00009F4B7C08637910524F483379105B9F15F
:1008C00007C28837910509F4AAC002C280E190E00E
:1008D000482A592AE0E2F0E04E2A5F2A15C220E8B1
:1008E00030E0422A532A10C280E490E0482A592A74
:1008F0000BC2E8E0F0E04E2A5F2A1A8A05C224E023
:1009000030E0422A532A00C20F2EFFE3AF2EF02D13
:100910007A940F2EF3E66F2EF02D65C1ED85FE85DE
:10092000CF0102968D879E87A0807A945CC1ED8569
:10093000FE859F012E5F3F4F2D873E87A080B180AF
:1009400043FE0BC03A89832F992787FD9095BC0100
:10095000C5010E94E8068F8707C0F50101900020BD
:10096000E9F73197EA19EF878F85781A3CC1ED8551
:10097000FE859F012E5F3F4F2D873E87A080B1806F
:1009800043FE0BC03A89832F992787FD9095BC01C0
:10099000C5010E94F3068F8704C0C5010E94DF06CF
:1009A0008F878F85781A1FC142FE0CC0ED85FE85AA
:1009B0009F012C5F3F4F2D873E87208131814281EF
:1009C00053810DC0ED85FE85CF0102968D879E87F0
:1009D000808191819C01442737FD4095542F590116
:1009E0006A01552364F4E2E0F0E04E2A5F2AD094D5
:1009F000C094B094A094A11CB11CC11CD11C2FEBBD
:100A00003FEF422253222CC038E03F870AC080E4E7
:100A100090E0482A592A0F2EF8E76F2EF02D90E12A
:100A20009F8742FE0CC0ED85FE859F012C5F3F4FE6
:100A30002D873E8720813181428153810BC0ED8516
:100A4000FE85CF0102968D879E87808191819C01D2
:100A50004427552759016A01EFECFFEF4E225F2230
:100A60009E012F5F3F4F288B398B3F85E32EFF245C
:100A700000271127C601B501A80197010E941D0793
:100A8000DC01CB01E889F98980838A301CF0860D6E
:100A9000815204C0E889F9898081805DE889F989FB
:100AA0008193E88BF98BC601B501A80197010E94DB
:100AB0001D0759016A012115310541055105D1F67E
:100AC000CE010196A888A81AC20182739070892B62
:100AD00009F07A9446FE0FC0872D992787FD9095DF
:100AE000FF85F03131F40F2EFEEF7F2EF02D780EC2
:100AF00002C0782E7A9443FE12C08A89282F3327A9
:100B000027FD30958A2D9927821793072CF0E7EF60
:100B1000FFEF4E225F2203C0FA89FA19FA8B43FED7
:100B200003C02A89721A01C07A18C20180789170B4
:100B3000892B69F4872D7A9418164CF4B40180E25D
:100B400090E00E94AC06872D7A941816BCF341FE03
:100B500006C0B4018DE290E00E94AC060FC044FED6
:100B600006C0B4018BE290E00E94AC0607C045FECF
:100B700005C0B40180E290E00E94AC0646FE0FC0C2
:100B8000B40180E390E00E94AC063F85303139F437
:100B9000B401862D992787FD90950E94AC06852D7E
:100BA000992780FF0DC0872D7A9418164CF4B40154
:100BB00080E390E00E94AC06872D7A941816BCF36F
:100BC00043FE11C08A89982F91509A8B18165CF4B5
:100BD000B40180E390E00E94AC068A89E82FE150DE
:100BE000EA8B1816ACF347FC0DC0872D7A941816C3
:100BF0004CF4B40180E290E00E94AC06872D7A9418
:100C00001816BCF3F3E66F1641F48A2DB401992748
:100C100087FD90950E94AC064BC023E76216B9F49D
:100C20003F8531503F873F3F09F442C0F501808145
:100C30000894A11CB11CB401992787FD90950E94CE
:100C4000AC068F8581508F878F3F81F731C093E548
:100C50006916A1F4EF85E150EF87EF3F49F1F50107
:100C60008491B40199270E94AC060894A11CB11C80
:100C7000FF85F150FF87FF3F91F71AC0CE01019623
:100C8000288939898217930799F08E010F5F1F4FCA
:100C9000E889F9898291E88BF98BB401992787FD5E
:100CA00090950E94AC06288939890217130781F7AD
:100CB00047FE15C0872D7A9418168CF4B40180E293
:100CC00090E00E94AC06872D7A941816BCF307C0FA
:100CD000B401862D992787FD90950E94AC06442487
:100CE000552412C035E2631641F44424552443943C
:100CF0001A8A7A888AE08F8707C0B401862D9927DF
:100D000087FD90950E94AC06F401838183FF03C0A8
:100D1000F101649002C0F1016080662009F04BCDC2
:100D2000F4018681978162960FB6F894DEBF0FBEFC
:100D3000CDBFDF91CF911F910F91FF90EF90DF908A
:100D4000CF90BF90AF909F908F907F906F905F906B
:100D50004F903F902F9008950F931F93CF93DF9361
:100D60008C01EB018B81992781FF22C082FF14C087
:100D70002E813F818C819D81281739073CF4E881C1
:100D8000F9810193E883F9832E813F812F5F3F4FE3
:100D90002E833F83C8010EC0E885F985802F099511
:100DA000892B31F4AE81BF811196AE83BF83F2CF20
:100DB0008FEF9FEFDF91CF911F910F910895FC016D
:100DC00005900020E9F7809590958E0F9F1F08955C
:100DD000FC016150704001900110D8F7809590950A
:100DE0008E0F9F1F0895FC01615070400590011007
:100DF000D8F7809590958E0F9F1F0895629FD00120
:100E0000739FF001829FE00DF11D649FE00DF11DC5
:100E1000929FF00D839FF00D749FF00D659FF00D74
:100E20009927729FB00DE11DF91F639FB00DE11D61
:100E3000F91FBD01CF0111240895A1E21A2EAA1BAA
:100E4000BB1BFD010DC0AA1FBB1FEE1FFF1FA2177A
:100E5000B307E407F50720F0A21BB30BE40BF50B77
:100E6000661F771F881F991F1A9469F76095709500
:0E0E7000809590959B01AC01BD01CF010895C6
:060E7E0025386C64000041
:00000001FF
